:020000040800F2
:10000000404500204D010008951800081511000812
:1000100091180008C3020008F92A00080000000037
:10002000000000000000000000000000071B0008A6
:10003000330B000800000000630100086D1C00087D
:1000400067010008670100086701000867010008F0
:1000500067010008670100086701000867010008E0
:1000600067010008670100086701000867010008D0
:100070007D090008670100087F0900086701000882
:1000800067010008670100086701000867010008B0
:1000900067010008670100086701000867010008A0
:1000A0006701000867010008670100086701000890
:1000B0006701000867010008670100086701000880
:1000C0006701000867010008670100086701000870
:1000D00067010008B1250008B9250008C1250008FE
:1000E0006701000867010008670100086701000850
:1000F0006701000867010008670100086701000840
:10010000670100086701000867010008670100082F
:10011000670100086701000867010008670100081F
:10012000670100086701000867010008670100080F
:10013000DFF80CD000F094F8004800470D320008BA
:100140004045002080F3088870470000064880473B
:1001500006480047FEE7FEE7FEE7FEE7FEE7FEE7AC
:10016000FEE7FEE7FEE7FEE7951C00083101000808
:1001700040EA01039B0703D009E008C9121F08C029
:10018000042AFAD203E011F8013B00F8013B521EA9
:10019000F9D27047D2B201E000F8012B491EFBD220
:1001A00070470022F6E710B513460A460446194682
:1001B000FFF7F0FF204610BD421E12F8013F002B52
:1001C000FBD111F8013B02F8013B002BF9D170473C
:1001D00010B5002200E0521C835C8C5CA34201D16C
:1001E000002BF8D1D8B2E1B2401A10BD034611F885
:1001F000012B00F8012B002AF9D1184670472DE990
:10020000F05F0546002092469B468846064681469A
:1002100040241BE0284641464746224600F041F86C
:1002200053465A46C01A914110D3114618462246E9
:1002300000F028F82D1A67EB01084F4622460120EE
:10024000002100F01FF817EB00094E41201EA4F119
:100250000104DFDC484631462A464346BDE8F09FAC
:10026000064C074D06E0E06840F0010394E8070003
:1002700098471034AC42F6D3FFF75EFFE43700082E
:1002800004380008202A04DB203A00FA02F100209A
:1002900070479140C2F1200320FA03F319439040C4
:1002A0007047202A04DB203A21FA02F0002170472F
:1002B00021FA02F3D040C2F12002914008431946CE
:1002C000704700BFFEE700002DE9F05F05460E46CF
:1002D00006EB460000EBC60105F1080000EB8100CB
:1002E000D0F8249006EB460000EBC60105F10800AB
:1002F00000EB8100D0F828B00027B846BA4623E0CA
:10030000A9EB0800B0F5006F02D34FF4006406E0DB
:10031000A9EB080084B20AF1010000F0FF0A0B4AC1
:100320005A44D1190A4A5068224603F003F8084893
:1003300021464268384600F0DFF8BAF1000F01D0DC
:10034000BDE8F09FA0442744DAE700000010200039
:100350004C0000202DE9F04F85B007464FF4805542
:100360004FF000090DE009EB490000EBC90107F16E
:10037000080000EB8100406A054409F1010000F02B
:10038000FF0978684845EED800260024A24639E0E7
:10039000281BB0F5006F02D34FF4006806E0281B5D
:1003A0001FFA80F80AF1010000F0FF0A18494246DE
:1003B000486818493144491C02F0BCFF14494246C0
:1003C0004868314603F02CF84644444464206043B6
:1003D000B0FBF5F000F0FF0B019858450ED0CDF8BA
:1003E00004B064206043B0FBF5F002460AA100901F
:1003F00002A802F041FC02A801F094F8BAF1000F43
:1004000000D000E0C4E700BF05B0BDE8F08F0000F9
:100410004C000020FFFF1F00436F707920256420EF
:100420000D0A000070B5ADF5786D284800780228F7
:1004300002D00DF5786D70BD6E464FF478624FF4C2
:100440000011304602F076FF2149009888423BD1E6
:10045000002220A1684600F0BCFD0546681C00B9DA
:10046000E7E7E9B26846FFF72FFF6846FFF772FF3C
:10047000002412E004EB440000EBC40102A800EBEE
:100480008100806A00F5805004EB440101EBC40256
:1004900002A901EB82018862641C0198A042E9D89C
:1004A0004FF478620021304602F0BAFF0B4800900A
:1004B0000422D104304602F0B3FF09480090042220
:1004C0000021304602F0ACFF00BFB2E74C00002034
:1004D000A9CBED9F485331350D0A000087D52F7504
:1004E000F8DEBC8A02200249087002484860704762
:1004F0004C000020B60000202DE9F04104460D46D6
:100500001646002704F0010010B10020BDE8F0817C
:10051000AAB203496018314602F06CFB0120F5E7EE
:10052000004000082DE9F04104460D4616463346CA
:100530002A462146044801F05FF907463946024839
:1005400002F0C4FABDE8F0815A21002010B5044839
:1005500001F080F904462146014802F0B7FA10BDC7
:100560005A2100202DE9F04FB5B00646B246DAF820
:100570000000E049884204D04FF0FF3035B0BDE8BC
:10058000F08F9AF80400952802D06FF00100F5E78B
:100590009AF805B0BAF818000290BBF1030F7CD1AD
:1005A00040F682710298884202D06FF00300E5E7BE
:1005B0003546B5F89A9F4FF4786205F11A0100208C
:1005C00002F0B4FD8046C84502D06FF00400D5E7C4
:1005D000D5F81E0008B90020D0E705F11A0000F098
:1005E00013FCC5490880D5F81E000988884209D83F
:1005F000D5F81E00C1494860C148086000F0F8FB0A
:100600000020BBE7D5F81E00BC494860D5F81E3075
:10061000DFF8E4C2BCF800C0A3EB0C034FF02C0CD5
:1006200003FB0CF2B44B1B8803EB430C0CEBC30C29
:1006300005F1220303EB8C01AF4B1B8803EB430C4A
:100640000CEBC30CAD4B083303EB8C00FFF790FDB4
:100650000020AC490860A9484268ABA103A802F099
:100660000BFB03A800F05EFFA348008800EB4001ED
:1006700001EBC001A148083000EB8100406A009006
:100680009D48008800EB400101EBC0019B48083009
:1006900000EB81039848028800E010E09FA103A8C6
:1006A00002F0EAFA03A800F03DFF4FF480529548AB
:1006B000016891480088FFF735FF01205EE7BBF134
:1006C000040F75D13446D4F83E10B4F8460000EB60
:1006D000400202EBC0028948083000EB8200406A09
:1006E00081420AD1A06C87490968884205D1B4F8D3
:1006F00046008149098888420DD08EA000F012FF83
:100700004FF480527F4801687B480088FFF70AFF5A
:100710006FF0050032E7E76CBF1E3A4604F1500166
:10072000002002F003FD814604F15000791C405C7A
:100730004FEA002804F15000C05D40441FFA80F8E1
:10074000C8450DD084A000F0EDFE4FF480526D48F6
:10075000016869480088FFF7E5FE6FF007000DE7C4
:10076000BAB26548008800EB400303EBC00363485E
:10077000083000EB8300806A624B1B68C11804F1EB
:10078000500002F04DFE5F4800683918D4F83E0072
:1007900081427DD359484068401E574909888842A4
:1007A00007D157485549086000F022FB0020E5E6D4
:1007B0009DE05148008800F093FA50BB0020514959
:1007C00008604D48008800EB400101EBC0014B4838
:1007D000083000EB8100406A00904748008800EB39
:1007E000400101EBC0014548083000EB810342485D
:1007F00002884AA103A802F03FFA03A800F092FE83
:100800004FF480523F4801683B480088FFF78AFE5A
:100810006BE039480088401C37490880084600884A
:10082000401E00EB400101EBC0013448083000EBF2
:100830008100816A30480088401E00EB400202EBD4
:10084000C0022E48083000EB8200406A01442A486A
:10085000008800EB400202EBC0022848083000EBA1
:10086000820081620020274908602348008800EB4D
:10087000400101EBC0012148083000EB8100406AD3
:1008800000901D48008800EB400101EBC00100E032
:1008900015E01A48083000EB8103174802881FA1B1
:1008A00003A802F0E9F903A800F03CFE4FF48052DF
:1008B0001448016810480088FFF734FE15E011481D
:1008C000006838440F490860084629A1026803A857
:1008D00002F0D2F903A800F025FE4FF48052094837
:1008E000016805480088FFF71DFE022046E600BFAC
:1008F00044E60000504354417C000020BE2100200B
:10090000F8DEBC8A800000205246696C6520436F87
:10091000756E743D256C750D0A0000005246696CB9
:10092000655B25645D3A257320206C656E3D256C02
:10093000750D0A0046696C65204C656E6774682009
:100940006F72204F6666736574206572726F7221D4
:100950005265444F210D0A00436865636B20435282
:1009600043206572726F72215265444F210D0A0057
:100970006F66667365743D25640D0A0070477047A5
:1009800021B1026842F00102026004E002684FF601
:10099000FE731A400260704701684FF6FE72114004
:1009A00001600021016041608160C1604B49884263
:1009B00008D14A490839496841F00F01474A083AC5
:1009C00051608AE045491431884208D143490839C9
:1009D000496841F0F001414A083A51607DE03F49E1
:1009E0002831884208D13D490839496841F470618D
:1009F0003A4A083A516070E038493C31884208D19F
:100A000036490839496841F47041344A083A51601E
:100A100063E032495031884208D130490839496889
:100A200041F470212D4A083A516056E02B49643157
:100A3000884208D129490839496841F47001274A98
:100A4000083A516049E025497831884208D1234964
:100A50000839496841F07061204A083A51603CE029
:100A60001F49884206D1011F096841F00F01021F8A
:100A7000116032E01A491431884208D11849091F1F
:100A8000096841F0F001164A121F116025E014496F
:100A90002831884208D11249091F096841F4706160
:100AA0000F4A121F116018E00D493C31884208D1ED
:100AB0000B49091F096841F47041094A121F11606E
:100AC0000BE007495031884207D10549091F0968E1
:100AD00041F47021024A121F116070470800024061
:100AE000080402401AB103680B43036002E0036884
:100AF0008B430360704710B50022026847F6F0731D
:100B00009A430C6A8B6823430C6923434C69234343
:100B10008C692343CC6923434C6A23438C6A234367
:100B20001A430260CB6843600B6883604B68C36004
:100B300010BD704710B5024607E0002101E04B1CD4
:100B400099B241F270739942F9DB131EA2F10104CC
:100B5000A2B2F2D110BD4FF0E0231A6900210CE0DF
:100B600008E04FF0E0231B69934203D04FF0E023ED
:100B70001A6900E0F5E700BF491C8142F0DB7047CD
:100B800001461CE000BF00BF00BF00BF00BF00BFA8
:100B900000BF00BF00BF00BF00BF00BF00BF00BF5D
:100BA00000BF00BF00BF00BF00BF00BF00BF00BF4D
:100BB00000BF00BF00BF00BF00BF00BF00BF0A1ED4
:100BC000A1F1010399B2DDD17047000030B50446B0
:100BD00004254FF4302000F06FF80546042D17D19E
:100BE0000C48006940F002000A4908610846446167
:100BF000006940F0400008614FF4302000F05CF8DC
:100C000005460448006941F6FD7108400149086144
:100C1000284630BD0020024004200B49C96801F07D
:100C2000010109B101200EE00749C96801F0040182
:100C300009B1022007E00449C96801F0100109B1B7
:100C4000032000E0042070470020024003480069B0
:100C500040F0800001490861704700000020024018
:100C600070B504460D460426F00200F025F806464D
:100C7000042E11D10948006940F0010007490861BC
:100C80002580F00200F018F806460448006941F695
:100C9000FE71084001490861304670BD00200240E5
:100CA000024803494860034848607047230167458C
:100CB00000200240AB89EFCD00B502460423FFF7C8
:100CC000ABFF034603E0FFF7A7FF0346521E012BCD
:100CD00001D1002AF7D102B90523184600BD000052
:100CE0002DE9F043ADF26C4D064606EB460000EBF5
:100CF000C6012B4800EB8100D0F8248006EB4600AB
:100D000000EBC601264800EB8100D0F828904F4642
:100D100045460DF2044000F0A7FC20E0B5F5806FD9
:100D200011D94FF48062394601A802F003FB4FF459
:100D3000806201A90DF2044000F0A8FC07F580676D
:100D4000A5F580650BE0AAB2394601A802F0F2FAD7
:100D50002A4601A90DF2044000F098FC0025002D60
:100D6000DCD10DF2044000F017FC002413E006EB88
:100D7000460000EBC6010A4800EB81001430015D1B
:100D80000DF25C40005D814204D000200DF26C4DFC
:100D9000BDE8F083641C102CE9DB0120F6E70000BD
:100DA000C621002010B500F017F80948006809496D
:100DB00088420BD04FF478610548FFF7F2F90548F7
:100DC0000349086000F014F8012010BD0020FCE782
:100DD000BE210020F8DEBC8A10B5044C4FF47862C6
:100DE0000021204602F0A6FA10BD0000BE2100201E
:100DF00010B5044C4FF478620021204602F010FB3D
:100E000010BD0000BE21002070B50646002446E05B
:100E100004EB440000EBC401254800EB8100416A6B
:100E200004EB440000EBC40206F1080000EB820072
:100E3000406A814200D037E0002516E004EB440010
:100E400000EBC4011A4800EB81001430415D04EB53
:100E5000440000EBC40206F1080000EB82001430ED
:100E6000405D814200D002E06D1C102DE6DB00BF2A
:100E7000102D00D018E004EB440202EBC40306F18D
:100E8000080202EB830104EB440202EBC403084AAC
:100E900002EB8300FFF79CF900B105E0641C0448F5
:100EA00008384068A042B3D800BF204670BD00009B
:100EB000C62100202DE9F041024600250026002031
:100EC00000230024002791F803C00CF00F0591F8CF
:100ED00003C00CF0100CBCF1000F03D091F802C05D
:100EE0004CEA050591F800C0BCF1000F31D0146840
:100EF00000202BE04FF0010C0CFA00F3B1F800C019
:100F00000CEA03069E4220D183004FF00F0C0CFA2E
:100F100003F7BC4305FA03FC4CEA040491F803C050
:100F2000BCF1280F06D14FF0010C0CFA00FCC2F8FE
:100F300014C00AE091F803C0BCF1480F05D14FF08E
:100F4000010C0CFA00FCC2F810C0401C0828D1D3D8
:100F50001460B1F800C0BCF1FF0F34DD546800200C
:100F60002EE000F1080C4FF0010808FA0CF3B1F87C
:100F700000C00CEA03069E4221D183004FF00F0C03
:100F80000CFA03F7BC4305FA03FC4CEA040491F89D
:100F900003C0BCF1280F05D100F1080C08FA0CF8C9
:100FA000C2F8148091F803C0BCF1480F07D100F1DA
:100FB000080C4FF0010808FA0CF8C2F81080401C29
:100FC0000828CED35460BDE8F081416170470161CB
:100FD00070472DE9F04105468846174600246EE02B
:100FE00057B105F1080108194146FFF7F1F800284B
:100FF00063D12046BDE8F08100265BE004EB4400AD
:1010000000EBC40105F1080000EB8100805D2E2893
:101010004ED1C6F11400032849DB04EB440000EB79
:10102000C40105F1080000EB8101701C085C422836
:101030000BD004EB440000EBC40105F1080000EB09
:101040008101701C085C622832D104EB440000EB83
:10105000C40105F1080000EB8101B01C085C4928BF
:101060000BD004EB440000EBC40105F1080000EBD9
:101070008101B01C085C69281AD104EB440000EB24
:10108000C40105F1080000EB8101F01C085C4E284A
:101090000BD004EB440000EBC40105F1080000EBA9
:1010A0008101F01C085C6E2802D12046A2E703E013
:1010B000701CC6B2142EA1DB00BF601CC4B26868ED
:1010C000A0428DD84FF0FF3094E73EB558246846D3
:1010D00000F010F8002503E01DF8050044406D1CE9
:1010E0000C2DF9DB04B95824FF2C00D185242046AF
:1010F0003EBD00000021064A00BF05E013780370E2
:10110000401C521C4B1CD9B20C29F7DB7047000065
:10111000E8F7FF1F0948C08808498988084307493C
:101120004988084305490988084305490880084655
:10113000018804A001F090FD00BFFEE70000002040
:10114000080000200D0A5B4846483D253034785D94
:101150000D0A00002DE9F043ADF6740D07468846F0
:101160004FF000090DF60C0000F07EFA0025002477
:1011700017E02C49601800F0C3FC064628466D1C99
:1011800003A90E54320A28466D1C0A54B5F5006FA7
:1011900006D14FF400620DF60C0000F077FA00253E
:1011A000A41CBC42E5D32DB12A4603A90DF60C00C0
:1011B00000F06CFA0DF60C0000F0EEF93A461AA1B8
:1011C00003A801F059FD00240BE00DF66400025D58
:1011D0001AA101A801F050FD01A903A8FEF7ECFF38
:1011E000641C102CF1DB17A103A8FEF7E5FF03A890
:1011F00000F098F9002408E018F804100DF66400D7
:10120000005D814200D002E0641C102CF4DB00BFC2
:10121000102C04DA00200DF6740DBDE8F0830120D7
:10122000F9E700000040000846696C6553697A657B
:101230003D256420204D44353D00000025303258C6
:10124000000000000D0A000070B504460D46074876
:1012500084420AD14FF400622946054800F06CFA36
:1012600006463146024801F031FC70BD50435441FE
:101270005A21002070B504460548844207D105482C
:1012800000F08CFA05462946024801F01FFC70BDAB
:10129000504354415A2100202DE9F04FA1B080461F
:1012A000444620687A49884208D0206879498842B3
:1012B00004D04FF0FF3021B0BDE8F08F20798028B6
:1012C00002D06FF00100F6E773A11DA801F0D4FC75
:1012D000A11D1DA8FEF77CFF10B16FF00200EAE728
:1012E00094F805A0208B0190BAF1000F25D1019848
:1012F000142802D06FF00300DDE7C34610220BF183
:101300001A016648FEF734FFD846DBF82A00644924
:1013100008600846006810B96FF00400CBE70020B1
:1013200060490860604908606049086020685D495C
:101330000968FFF789FF0120BDE7BAF1020F7DD1EF
:101340004746002608E05548815D07F11A00805D98
:10135000814200D002E0761C102EF4DB00BF102E7C
:1013600008DA53A000F0DEF82068FFF783FF6FF083
:101370000500A0E7D7F82E50D7F82A000290022DDA
:101380000CD3484902980968884207D1454800684B
:10139000291843480068801C814208D949A000F000
:1013A000C1F82068FFF766FF6FF0060083E7AD1E07
:1013B0002A4607F13201002001F0B8FE814607F10C
:1013C0003200691C405C00021C9007F13200405D55
:1013D0001C99084480B21C901C9949450AD041A030
:1013E00000F0A0F820682F490968FFF72DFF6FF083
:1013F000070060E72068274988420DD1002609E0F0
:1014000007F13200805D3D490978484007F132011B
:101410008855761CAE42F3D307F1320229462148A3
:10142000006800F0A3F82148006828441F490860BC
:101430001C48006828441B49086000E026E01B485F
:10144000006817490968884210DB1449144800688D
:10145000FFF780FE40B92AA000F064F82068FFF78B
:1014600009FF6FF0080026E7002024E70D482AA1B5
:10147000026803A801F000FC03A800F053F82068FC
:1014800008490968FFF7E0FE022014E700BF12E7F1
:10149000464F54415043544130000000A600002004
:1014A000340000203C0000204000002038000020D4
:1014B0004D4435204D6F64696679215265444F2152
:1014C0000D0A00004C656E677468206F72204F66CD
:1014D00066736574206572726F72215265444F2184
:1014E0000D0A0000436865636B2043524320657218
:1014F000726F72215265444F210D0A002C000020AA
:10150000436865636B204D4435206572726F7221AC
:101510005265444F210D0A004842443D25640D0A9E
:101520000000000070B505462C460A20FFF713FBAB
:101530000BA001F091FB0BE021780B4801F02FF993
:1015400000BF4021084801F05DF80028F9D0641C74
:1015500020780028F0D10A20FFF7FDFA70BD0000C6
:101560005B4941505D000000003801402DE9F04129
:1015700004460D461646002704F0010010B1002075
:10158000BDE8F081AAB203496018314601F032FB90
:101590000120F5E7004000082DE9F04190B0044635
:1015A00020680E9060680F902088C0F3C507382F20
:1015B00002DAC7F1380001E0C7F178008046424600
:1015C0002849204600F062F80026002518E004F1C2
:1015D0001800E91C405C020604F11800A91C405CDC
:1015E00042EA004204F11800691C405C42EA002013
:1015F00004F11801495D08434DF82600761C2D1DA5
:101600000E2EE4D3694604F1080000F0AFFB00267B
:10161000002521E004F1080010F826105030415553
:10162000503830F82600C0F3072204F15800691C36
:101630004254503850F82600C0F3074204F15800D5
:10164000A91C4254503850F82600000E04F15801ED
:10165000EA1C8854761C2D1D042EDBD310B0BDE887
:10166000F0810000A23500080021416001600549B9
:101670008160054AC260CA430261034AD2434261A3
:10168000704700000123456789ABCDEF2DE9F0439A
:1016900091B004460F4615462088C0F3C50920685E
:1016A00000EBC5002168884202D26068401C60607F
:1016B000206800EBC5002060606800EB557060603A
:1016C00033E017F8012B484609F1010904F118012C
:1016D0000A54B9F1400F28D14FF0000800261AE053
:1016E00004F11800F11C405C020604F11800B11C62
:1016F000405C42EA004204F11800711C405C42EA7E
:10170000002004F11801895D084301A941F828006F
:1017100008F10108361DB8F1100FE1D301A904F159
:10172000080000F023FB4FF00009281EA5F1010579
:10173000C7D111B0BDE8F0832DE9F04104460E4653
:101740001746254632212846FEF72BFD0F48286014
:1017500080202871022068710DA1A81D01F08CFA6B
:101760000C480088401C80B20A490880E882182092
:1017700028831022084905F11A00FEF7F9FCC5F884
:101780002A60C5F82E703220BDE8F08150435441E4
:101790003000000030000020A600002070B5044694
:1017A00025462C212846FEF7FCFC0D4828608020A9
:1017B0002871002068710BA1A81D01F05DFA0A488C
:1017C0000078E8821220288308A105F11A00FEF7AC
:1017D0000DFD00206885074908802C2070BD0000A1
:1017E00050435441300000002C0000204E554C4C1A
:1017F00000000000300000202DE9F04104460E46B4
:1018000017469846254650212846FEF7CAFC0F4841
:10181000286095202871042068710020E882362015
:101820002883A5F8466006EB460000EBC602084890
:1018300000EB82012C2205F11A00FEF799FCC5F895
:101840004C80AF645020BDE8F0810000504354410B
:10185000C621002070B50446254622212846FEF701
:10186000A0FC094828609520287103206871002099
:10187000E882082028835A20A8831420688303481C
:10188000C5F81E00222070BD5043544100F01F00D7
:1018900000BFFEE77047000070B5002100230F2253
:1018A000C47804B3154C246804F4E064C4F5E0641F
:1018B000210AC1F10403CA40447804FA03F1847890
:1018C0001440214309010E4C0678A155047804F018
:1018D0001F050124AC4005786D11AD0005F1E02530
:1018E000C5F8004109E0047804F01F050124AC406C
:1018F000044D0678761145F8264070BD0CED00E0E9
:1019000000E400E080E100E002490143024A116086
:10191000704700000000FA050CED00E0044909786A
:10192000044A1170024908700121034A517170473D
:1019300017000020180000201000002029B1064ADE
:1019400052690243044B5A6104E0034A52698243DC
:10195000014B5A61704700000010024029B1064A4D
:1019600092690243044B9A6104E0034A92698243FC
:10197000014B9A61704700000010024030B5002111
:101980000022002400232D4D6D6805F00C0121B1CB
:10199000042905D0082923D105E0294D056022E05E
:1019A000284D05601FE0254D6D6805F47012234D2C
:1019B0006D6805F48034022505EB92421CB9224D76
:1019C000554305600BE01D4D6D6805F400351DB1F4
:1019D0001E4D5543056002E01A4D5543056002E077
:1019E000174D056000BF00BF144D6D6805F0F00194
:1019F0000909174D6B5C0568DD4045600F4D6D684A
:101A000005F4E061090A124D6B5C4568DD408560B4
:101A10000A4D6D6805F46051C90A0D4D6B5C45684F
:101A2000DD40C560054D6D6805F44041890B094DE9
:101A30006B5CC568B5FBF3F5056130BD0010024075
:101A400000127A00001BB70000093D00808D5B008A
:101A5000540000206400002021B1028842F04002BE
:101A6000028004E002884FF6BF731A40028070477C
:101A70000246002013890B400BB1012000E000203A
:101A800070470146888970478181704710B50022F0
:101A9000028802F441520B884C8823438C882343EC
:101AA000CC8823430C8923434C8923438C892343CB
:101AB000CC8923431A430280838B4FF2FF74234067
:101AC00083830B8A038210BD10B5044600BF022138
:101AD0000A48FFF7CDFF0028F9D021460748FFF755
:101AE000D3FF00BF01210548FFF7C2FF0028F9D04E
:101AF0000248FFF7C6FFC0B210BD00000030014031
:101B0000014608887047704710B500F001F810BD15
:101B10000CB50020019000903148006840F48030FE
:101B20002F49086000BF2E48006800F40030009084
:101B30000198401C0190009818B90198B0F5A06F69
:101B4000F1D12748006800F4003010B10120009066
:101B500001E000200090009801283FD12148006852
:101B600040F010001F4908600846006820F003009C
:101B700008600846006808601948406818494860CD
:101B80000846406848600846406848600846406823
:101B900020F47C1048600846406840F430204860DB
:101BA0000846006840F08070086000BF0C4800687C
:101BB00000F000700028F9D00948406820F00300C8
:101BC000074948600846406840F00200486000BF8E
:101BD0000348406800F00C000828F9D10CBD000053
:101BE000001002400020024030B502460B46194664
:101BF000144607E008782578A84201D0012030BDBE
:101C0000491C641C08780028F4D100BFF7E70000E5
:101C100010B500201049086010490860104800788D
:101C2000122806D0342805D0562807D0782810D19D
:101C300007E00EE00B48FFF71DFB0AE0FEF786FC0D
:101C400007E0FEF7EFFB0848FFF76CFC01F09EFA97
:101C500000BF00BF10BD0000200000201C000020BD
:101C600017000020504354419435000801200749D3
:101C7000C87007480068401C05490860322804DB2A
:101C80000020086001200149087170471000002001
:101C90000C00002010B51348006840F00100114905
:101CA000086008464068104908400E4948600846E8
:101CB00000680E4908400B4908600846006820F497
:101CC000802008600846406820F4FE0048604FF419
:101CD0001F008860FFF718FF4FF00060044908609C
:101CE00010BD0000001002400000FFF8FFFFF6FEEC
:101CF00008ED00E010B517480068401C20B11548F9
:101D00000068401C1349086013480078122806D068
:101D100034280CD056280BD0782818D109E00D486B
:101D20000068012802D17820FFF7F8FD0FE00EE0EF
:101D30000DE008480068042800D210BD054800786E
:101D400000F0010010B105A0FFF7ECFB00BF00BFE1
:101D500000BFF2E720000020170000204E6F204156
:101D60007070210D0A00000070470000F0B50546B4
:101D70000C4628686968AA68EB6801EA020623EA4B
:101D800001073E4327683E44FE4F3E443044C601AF
:101D900046EA5060084400EA010622EA00073E4392
:101DA00067683E44F84F3E4433441E0346EA1353EB
:101DB000034403EA000621EA03073E43A7683E44C2
:101DC000F24F3E443244560446EAD2321A4402EA02
:101DD000030620EA02073E43E7683E44EC4F3E44D8
:101DE00031448E0546EA9121114401EA020623EAB4
:101DF00001073E4327693E44E64F3E443044C60156
:101E000046EA5060084400EA010622EA00073E4321
:101E100067693E44E04F3E4433441E0346EA135391
:101E2000034403EA000621EA03073E43A7693E4450
:101E3000DA4F3E443244560446EAD2321A4402EAA9
:101E4000030620EA02073E43E7693E44D44F3E447E
:101E500031448E0546EA9121114401EA020623EA43
:101E600001073E43276A3E44CE4F3E443044C601FC
:101E700046EA5060084400EA010622EA00073E43B1
:101E8000676A3E44C84F3E4433441E0346EA135338
:101E9000034403EA000621EA03073E43A76A3E44DF
:101EA000A6F524464F3E3244560446EAD2321A443E
:101EB00002EA030620EA02073E43E76A3E44BB4FBC
:101EC0003E4431448E0546EA9121114401EA02065E
:101ED00023EA01073E43276B3E44B54F3E4430445E
:101EE000C60146EA5060084400EA010622EA0007FB
:101EF0003E43676B3E44AF4F3E4433441E0346EAC5
:101F00001353034403EA000621EA03073E43A76B89
:101F10003E44A94F3E443244560446EAD2321A4463
:101F200002EA030620EA02073E43E76B3E44A34F62
:101F30003E4431448E0546EA9121114401EA0306EC
:101F400022EA03073E4367683E449D4F3E443044C7
:101F5000460146EAD060084400EA020621EA020788
:101F60003E43A7693E44974F3E4433445E0246EAEF
:101F7000D353034403EA010620EA01073E43E76A1C
:101F80003E44914F3E443244960346EA92421A44FC
:101F900002EA000623EA00073E4327683E448B4FCF
:101FA0003E4431440E0546EA1131114401EA03066C
:101FB00022EA03073E4367693E44854F3E4430446E
:101FC000460146EAD060084400EA020621EA020718
:101FD0003E43A76A3E447F4F3E4433445E0246EA96
:101FE000D353034403EA010620EA01073E43E76BAB
:101FF0003E44794F3E443244960346EA92421A44A4
:1020000002EA000623EA00073E4327693E44734F75
:102010003E4431440E0546EA1131114401EA0306FB
:1020200022EA03073E43676A3E446D4F3E44304414
:10203000460146EAD060084400EA020621EA0207A7
:102040003E43A76B3E44674F3E4433445E0246EA3C
:10205000D353034403EA010620EA01073E43E7683D
:102060003E44614F3E443244960346EA92421A444B
:1020700002EA000623EA00073E43276A3E445B4F1C
:102080003E4431440E0546EA1131114401EA03068B
:1020900022EA03073E43676B3E44554F3E443044BB
:1020A000460146EAD060084400EA020621EA020737
:1020B0003E43A7683E444F4F3E4433445E0246EAE7
:1020C000D353034403EA010620EA01073E43E769CC
:1020D0003E44494F3E443244960346EA92421A44F3
:1020E00002EA000623EA00073E43276B3E44434FC3
:1020F0003E4431440E0546EA1131114481EA02069C
:102100005E4067693E443E4F3E443044060146EA25
:102110001070084480EA01065640276A3E44394F51
:102120003E443344DE0246EA5353034483EA000646
:102130004E40E76A3E44344F3E443244160446EA79
:1021400012421A4482EA03064640A76B3E442F4FD0
:102150003E443144CE0546EA5121114481EA02064B
:102160005E4067683E442A4F3E443044060146EADA
:102170001070084480EA0106564027693E44254F06
:102180003E4449E078A46AD756B7C7E8DB702024FC
:10219000EECEBDC1AF0F7CF52AC68747134630A8E7
:1021A000019546FDD8988069AFF7448BBED75C890E
:1021B0002211906B937198FD8E4379A62108B44942
:1021C00062251EF640B340C0515A5E26AAC7B6E942
:1021D0005D102FD65314440281E6A1D8C8FBD3E783
:1021E000E6CDE121D60737C3870DD5F4ED145A4566
:1021F00005E9E3A9F8A3EFFCD9026F678A4C2A8DA1
:102200004239FAFF81F6718722619D6D0C38E5FD38
:1022100044EABEA4A9CFDE4B3344DE0246EA535360
:10222000034483EA00064E40E7693E449F4F3E4424
:102230003244160446EA12421A4482EA0306464031
:10224000A76A3E449A4F3E443144CE0546EA5121A6
:10225000114481EA02065E40676B3E44954F3E445E
:102260003044060146EA1070084480EA01065640F0
:1022700027683E44904F3E443344DE0246EA5353BF
:10228000034483EA00064E40E7683E448B4F3E44D9
:102290003244160446EA12421A4482EA03064640D1
:1022A000A7693E44864F3E443144CE0546EA51215B
:1022B000114481EA02065E40676A3E44814F3E4413
:1022C0003044060146EA1070084480EA0106564090
:1022D000276B3E447C4F3E443344DE0246EA535370
:1022E000034483EA00064E40E76B3E44774F3E448A
:1022F0003244160446EA12421A4482EA0306464071
:10230000A7683E44724F3E443144CE0546EA51210F
:10231000114461EA0306564027683E446D4F3E442F
:102320003044860146EA9060084460EA02064E4066
:10233000E7693E44684F3E4433449E0246EA935365
:10234000034463EA01064640A76B3E44634F3E44A4
:102350003244D60346EA52421A4462EA00065E401C
:1023600067693E445E4F3E4431444E0546EAD12102
:10237000114461EA03065640276B3E44594F3E44E0
:102380003044860146EA9060084460EA02064E4006
:10239000E7683E44544F3E4433449E0246EA93531A
:1023A000034463EA01064640A76A3E444F4F3E4459
:1023B0003244D60346EA52421A4462EA00065E40BC
:1023C00067683E444A4F3E4431444E0546EAD121B7
:1023D000114461EA03065640276A3E44454F3E4495
:1023E0003044860146EA9060084460EA02064E40A6
:1023F000E76B3E44404F3E4433449E0246EA9353CB
:10240000034463EA01064640A7693E443B4F3E440D
:102410003244D60346EA52421A4462EA00065E405B
:10242000676B3E44364F3E4431444E0546EAD12167
:10243000114461EA0306564027693E44314F3E4449
:102440003044860146EA9060084460EA02064E4045
:10245000E76A3E442C4F3E4433449E0246EA93537F
:10246000034463EA01064640A7683E44274F3E44C2
:102470003244D60346EA52421A4462EA00065E40FB
:10248000676A3E44224F3E4431444E0546EAD1211C
:1024900011442E6806442E606E680E446E60AE686D
:1024A0001644AE60EE681E44EE60F0BD604BBBF6B5
:1024B00070BCBFBEC67E9B28FA27A1EA8530EFD448
:1024C000051D880439D0D4D9E599DBE6F87CA21F34
:1024D0006556ACC4442229F497FF2A43A72394AB42
:1024E00039A093FCC3595B6592CC0C8F7DF4EFFF50
:1024F000D15D84854F7EA86FE0E62CFE144301A3D6
:10250000A111084E827E53F735F23ABDBBD2D72ACD
:1025100091D386EB08B540F224411D4800F07FF8C6
:1025200040B31B48008800901948001D00880090A7
:102530001848C06D41F25201081A00900021154858
:102540005830FEF71DFA1448007850B91349144862
:10255000009AFDF70DFE13490098088001200E49EE
:10256000087041F252000B49C865012109485830F2
:10257000FEF706FA08210C4800F044F8012806D1BD
:10258000034800F007F90821014800F01DF808BDD4
:102590000038014000000240100000200811002017
:1025A000B6000020440000200048004070477047FB
:1025B00010B5FFF7AFFF10BD10B5FFF7F7FF10BD67
:1025C00010B5FFF7F4FF10BD01F40072B2F5007F03
:1025D00000D100BFCA430280704721B1828942F412
:1025E0000052828104E082894DF6FF731A40828195
:1025F00070471AB1838A0B43838202E0838A8B433C
:102600008382704702460020B1F5007F00D100BFF1
:1026100013880B400BB1012000E00020704770B51B
:102620000246002400230025002040F66A16B1422D
:1026300000D100BFC1F3421501F01F03012606FAC5
:1026400003F3012D02D19689334006E0022D02D119
:10265000168A334001E0968A33400C12012606FAAE
:1026600004F41688344013B10CB1012000E00020BE
:1026700070BDF0B50346002400260025002040F67A
:102680006A17B94200D100BF1846C1F3421401F0E5
:102690001F06012707FA06F5012C01D10C3004E0D2
:1026A000022C01D1103000E014301AB107682F431A
:1026B000076002E00768AF430760F0BD2DE9F0470F
:1026C00086B005460E460024A24600BFA14600275C
:1026D000B08900B100BF2F462C8A4CF6FF70044031
:1026E000F08804432C82AC894EF6F3100440B08885
:1026F00031890843718908430443AC81AC8A4FF6A1
:10270000FF400440B0890443AC8201A8FFF736F9CA
:102710001F48874202D1DDF810A001E0DDF80CA0CF
:10272000A88900F4004040B10AEBCA0000EB0A108F
:1027300031684900B0FBF1F807E00AEBCA0000EB92
:102740000A1031688900B0FBF1F86420B8FBF0F0A2
:1027500004012009642101FB1089A88900F40040CC
:1027600040B1322000EBC900B0FBF1F000F00700EF
:10277000044308E0322000EB09106421B0FBF1F0C3
:1027800000F00F0004432C8106B0BDE8F087000084
:102790000038014001468888C0F308007047C1F343
:1027A000080282807047000000B58DB00121084604
:1027B000FFF7C4F82B48FEF7EFF82B4801902B48A1
:1027C0000290102003906420049000200590802047
:1027D000069000200790089009900A900B9001A99C
:1027E0002048FEF788F90E208DF8300003208DF880
:1027F000310002208DF8320001208DF833000CA842
:10280000FFF74AF8012202211648FEF76BF9002172
:102810001448FEF7B5F813481430FEF7BDF8124817
:102820000190134802900020039041F2520004905E
:1028300000200590802006900020079008900990C5
:102840004FF400500A9000200B9001A90548143065
:10285000FEF751F9012103481430FEF791F80DB04D
:1028600000BD000044000240043801405A2100200D
:102870000811002000B587B0012144F20400FFF7E1
:102880006DF84FF40070ADF8140018208DF81700A3
:1028900003208DF8160005A92E48FEF70BFB4FF418
:1028A0008060ADF8140004208DF8170003208DF827
:1028B000160005A92748FEF7FDFA4FF4E130019014
:1028C0000020ADF80800ADF80A00ADF80C00ADF836
:1028D00010000C20ADF80E0001A91F48FFF7EEFE16
:1028E00001211D48FFF779FE4FF4E060FFF70CF877
:1028F00025208DF8180000208DF819008DF81A0099
:1029000001208DF81B0006A8FEF7C6FF40211248E3
:10291000FFF75AFE002240F227710F48FFF7A9FE89
:10292000002240F225510C48FFF7A3FE012240F29D
:1029300024410948FFF79DFE012240210648FFF788
:1029400058FE002280210448FFF753FEFFF72CFFBA
:1029500007B000BD000801400038014010B53E48F6
:10296000007812281BD13DA14048FFF73DF930B94E
:102970003420FEF7D3FF3EA0FEF7D4FD0EE040A1C9
:102980003A48FFF731F930B95620FEF7C7FF40A0AB
:10299000FEF7C8FD02E043A0FEF7C4FD10BD2E48BF
:1029A0000078342804D02C480078562800D0F5E769
:1029B0002E48007850280BD12C484078432807D166
:1029C0002A488078542803D12848C078412800D06C
:1029D000E4E72648007980281AD134480188234842
:1029E000FEF75AFC044634B931A0FEF79BFD562091
:1029F000FEF794FFD2E714F1020F2ADA14F1060F62
:102A000027DD2EA0FEF78EFD7820FEF787FF20E061
:102A10001648007995281CD1244801881348FDF7F1
:102A2000A1FD04464CB922A0FEF77CFD7820FEF7FC
:102A300075FF012024490870B0E714F1020F08DA8D
:102A400014F1060F05DD1DA0FEF76CFD7820FEF7E2
:102A500065FF00BFA2E7000017000020444F574E5B
:102A60004C4F41445F41505000000000B600002030
:102A7000444F574E4C4F41445F4150500D0A0000A7
:102A8000444F574E4C4F41445F5246494C455300CA
:102A9000444F574E4C4F41445F5246494C45530DAD
:102AA0000A0000002D2D2D2D0D0A000044000020ED
:102AB000436F6D706C65746564210000494150205E
:102AC00053746F70210D0A004C00002070B505464C
:102AD0000E4600240BE0295D0648FFF760FE00BFAC
:102AE00040210448FFF78EFD0028F9D0641CB44251
:102AF000F1DB70BD0038014000BFFEE710B586B0C5
:102B000000F036F810211848FEF761FA0020ADF801
:102B100004004FF48270ADF806000020ADF8080004
:102B20000220ADF80A000120ADF80C004002ADF81B
:102B30000E000820ADF810000020ADF812000720AC
:102B4000ADF8140001A90948FEF7A0FF01210748CC
:102B5000FEF782FF4FF47A70FEF712F800F018FCCF
:102B60000446012006B010BD0008014000300140BD
:102B700008B501210420FEF7F1FE01210803FEF74C
:102B8000EDFE2020ADF8000003208DF80200182093
:102B90008DF8030069461548FEF78CF98020ADF8E2
:102BA000000069461148FEF785F94020ADF80000A5
:102BB00004208DF8030069460C48FEF77BF91020CD
:102BC000ADF800008DF8030069460848FEF772F979
:102BD0001020ADF800008DF8030069460448FEF7A8
:102BE00069F910210248FEF7F2F908BD000801401A
:102BF000001001402DE9F04705460E469046B5F11C
:102C0000006F02D31348854201D3BDE8F087C5F3B6
:102C10000A0000B1F9E7FEF743F82846FDF7D6FFB2
:102C20000746042F00D0F0E700240CE0315D601C63
:102C3000305C01EB00201FFA80F928194946FEF7A5
:102C40000FF8A01C84B24445F0DBFDF7FFFF00BF86
:102C5000DBE70000000004080FB4054B10B503A922
:102C6000044A029800F02CF810BC5DF814FB000038
:102C700069310008880000200FB4084B10B504A982
:102C800002AA039800F01CF8044602A9002000F0F4
:102C900048FA204610BC5DF814FB00002331000800
:102CA00002E008C8121F08C1002AFAD17047704715
:102CB000002001E001C1121F002AFBD17047000073
:102CC0002DE9FF4F8DB00F460546002606E025286A
:102CD0000BD0DDE90F1290476D1C761C2878002878
:102CE000F5D111B03046BDE8F08F0024A246A146D0
:102CF0000122EC4900E0044315F8013F203B02FAB1
:102D000003F00842F7D128782A2810D06FF02F025C
:102D10002878A0F13001092914D80AEB8A0102EBC6
:102D2000410144F0020400EB010A6D1CF0E701CF01
:102D30005FEA000A03D544F40054CAF1000A44F0E3
:102D400002046D1C28782E2817D115F8010F44F0C5
:102D500004042A280ED06FF02F022878A0F1300149
:102D600009290AD809EB890102EB410100EB0109AD
:102D70006D1CF2E757F8049B6D1C28786C280FD067
:102D800006DC4C2817D068280DD06A2814D104E03E
:102D9000742810D07A280FD10DE044F400140AE012
:102DA00044F4801401E044F440146978814202D173
:102DB00004F580146D1C6D1C2A786E2A1FD00CDC63
:102DC000632A31D004DC002A8BD0582A11D1A3E029
:102DD000642A68D0692A0CD165E0732A2ED004DCFD
:102DE0006F2A73D0702A04D19BE0752A6FD0782A9D
:102DF0006ED01046DDE90F129047761C50E1C4F307
:102E00000250022806D0032809D0042801CF09D097
:102E1000066045E101CFF117C0E9006140E101CF53
:102E200006803DE106703BE117F8040B8DF80000C9
:102E300000208DF80100EB46012003E057F804BBA9
:102E40004FF0FF3061074FF0000102D40DE008F1B0
:102E50000101884649450FDA8045F8DB1BF8081068
:102E60000029F4D108E008F1010188468142FADB2B
:102E70001BF808100029F6D1DDE90F23AAEB0800A2
:102E80008146214600F036F9304400EB080604E0A4
:102E9000DDE90F121BF8010B9047B8F10108F7D2DA
:102EA00021464846F7E00A21C4F302534FF0000BD5
:102EB0000891022B04D001CFC117032B09D00AE0DF
:102EC000FF1D27F00707F7E8020108E032E01FE0E6
:102ED00020E000B2C117042B01D140B2C117031E7C
:102EE00071F1000307DA4FF0000CD0EB0C006CEB33
:102EF00001012D2302E0230504D52B238DF8243076
:102F0000012303E0E30701D02023F7E7984658E0C8
:102F10000A2110E010210EE010204FF0000B089065
:102F20000CE010214FF0000B44F004044FF00809AE
:102F3000089103E008214FF0000B0891C4F30253FD
:102F4000022B04D001CF0021032B06D006E0FF1D89
:102F500027F00707F7E8020103E080B2042B00D155
:102F6000C0B24FF0000823072BD5702A07D0DDF838
:102F700020C08CF0100C5CEA0B0C05D00EE0402356
:102F80008DF82430012308E050EA010306D03023F5
:102F90008DF824308DF8252002239846DDF820C0D6
:102FA0008CF0080C5CEA0B0C0BD150EA010301D148
:102FB000630706D530238DF824304FF00108A9F1BE
:102FC0000109582A04D038A20B9208AA0A920BE0F1
:102FD0003AA2F9E75B46089AFDF711F90B9B9B5C57
:102FE0000A9A521E0A92137050EA0102F2D10A980C
:102FF000ADEB000000F1200B600702D524F4803413
:1030000001E04FF00109D94502DDA9EB0B0000E01A
:10301000002000EB0B0141440890AAEB010AE003F9
:1030200006D4DDE90F232146504600F063F806443C
:103030004FF0000908E009A911F80900DDE90F12B5
:10304000904709F10109761CC145F4DBE0030CD57A
:10305000DDE90F232146504600F04CF8064404E019
:10306000DDE90F1230209047761C0899481E089021
:103070000029F5DC08E00A980A990078491C0A91B1
:10308000DDE90F129047761CBBF10001ABF1010B9B
:10309000F1DC21465046DDE90F2300F019F8064423
:1030A0006D1C1BE6092801003031323334353637C8
:1030B0003839616263646566000000003031323384
:1030C0003435363738394142434445460000000024
:1030D0002DE9F041044600251E461746880404D415
:1030E00005E039462020B0476D1C641EF9D52846FE
:1030F000BDE8F0812DE9F041044600251E469046CA
:10310000C80301D5302700E02027880404D505E056
:1031100041463846B0476D1C641EF9D52846BDE8C7
:10312000F0810A68531C0B6010707047F0B50746B9
:103130000C461546002606E014F8011B384600F040
:1031400007F80746761CAE42F6D33846F0BD0000BD
:10315000024682EA0100C0B2024B33F8100080EA56
:1031600022207047E235000870B504460D46E1B2F2
:103170000548FFF714FB00BF40210348FFF742FA60
:103180000028F9D0204670BD0038014010B5024833
:1031900000F004F810BD00000040000810B504461F
:1031A000206814490840B0F1005F18D1002240F2B5
:1031B00024411148FFF75DFA002240210E48FFF735
:1031C00018FA00204FF0E021086160680B490860A0
:1031D0002068FCF7B7FF09480068804708E006E070
:1031E00007A0FEF79FF94FF47A70FDF7A3FCF7E70D
:1031F00010BD00000000FE2F0038014048000020F4
:103200004E6F204170700D0A00000000FFF732FB86
:10321000314800686422B0FBF2F1B1F1807F01D344
:1032200001201DE021F07F40401E4FF0E022506160
:1032300050170F22002807DA13071D0E274B00F046
:103240000F04241F1D5503E013071C0E244B1C54B0
:1032500000BF00204FF0E0229061072010610020A5
:1032600008B100BFFEE7FFF749FCFDF79BFDFDF746
:103270002CFF1C4908701C4800210160818081716D
:103280001220FEF74BFBFDF72DF924E016480078DD
:1032900048B1FFF763FB00201349087041F2520167
:1032A0001248FCF77EFF1048407920B100200E49FB
:1032B0004871FEF7ADFC0C48C07820B100200A49E7
:1032C000C870FEF751FD0848007920B1002006497A
:1032D0000871FEF70FFDD9E76800002018ED00E047
:1032E00000E400E02C00002010000020B6000020C8
:1032F00010B50446240300F0EDF800F087F8102123
:103300000B48FDF762FE2020FEF7DEFBC4F307400A
:10331000FEF7DAFBC4F30720FEF7D6FBE0B2FEF7B8
:10332000D3FB10210248FDF752FE00F06FF810BDEC
:10333000000801402DE9F04105460C4617461021D2
:103340001248FDF742FE0B20FEF7BEFBC4F3074018
:10335000FEF7BAFBC4F30720FEF7B6FBE0B2FEF7B8
:10336000B3FBFF20FEF7B0FB2870002605E0FF202E
:10337000FEF7AAFBA855701C86B2BE42F7DB1021EF
:103380000248FDF724FEBDE8F0810000000801407E
:103390002DE9F041002400250026002710210F48C8
:1033A000FDF713FE9F20FEF78FFBFF20FEF78CFB3F
:1033B0000546FF20FEF788FB0646FF20FEF784FB4C
:1033C000074610210548FDF702FE280440EA0620C2
:1033D00040EA07042046BDE8F081000000080140F3
:1033E00010B5002410210848FDF7EFFD0520FEF779
:1033F0006BFBFF20FEF768FB044610210248FDF737
:10340000E6FD204610BD00000008014010B500BFD9
:10341000FFF7E6FF00F001000028F9D110BD000021
:103420002DE9F04781460F4616464FEA1738C7F395
:103430000B0ACAF58054A64200DC344644E04FEA49
:1034400008314FF480522248FFF774FF002508E04E
:103450000AEB05001E49085CFF2800D003E0681C49
:1034600085B2A542F4DB00BFA54216DA4046FFF75D
:103470003FFF002507E019F8050005EB0A01144A93
:103480005054681C85B2A542F5DB4FEA08314FF471
:1034900080520F4800F02EF804E022463946484694
:1034A00000F028F8A64200D10FE008F101084FF023
:1034B000000AA1442744301B86B2B6F5805F02DDC6
:1034C0004FF4805400E03446B9E700BFBDE8F08710
:1034D0003E31002010B510210548FDF776FD06208D
:1034E000FEF7F2FA10210248FDF771FD10BD000051
:1034F000000801402DE9F04107460E461446F0B29F
:10350000C0F58075AC4200DC254612E02A46314603
:10351000384600F013F8AC4200D10BE02F442E44A3
:10352000601B84B2B4F5807F02DD4FF4807500E04B
:103530002546EBE700BFBDE8F08100002DE9F04132
:1035400006460C461746FFF7C5FF10211048FDF749
:103550003CFD0220FEF7B8FAC4F30740FEF7B4FAC8
:10356000C4F30720FEF7B0FAE0B2FEF7ADFA00258B
:1035700004E0705DFEF7A8FA681C85B2BD42F8DB76
:1035800010210348FDF723FDFFF740FFBDE8F08160
:103590000008014048532D4941502D563130330D1C
:1035A0000A00800000000000000000000000000091
:1035B000000000000000000000000000000000000B
:1035C00000000000000000000000000000000000FB
:1035D00000000000000000000000000000000000EB
:1035E00000000000C1C081C1400101C3C0038002CE
:1035F00041C201C6C006800741C70005C1C581C4DC
:10360000400401CCC00C800D41CD000FC1CF81CE54
:10361000400E000AC1CA81CB400B01C9C009800815
:1036200041C801D8C018801941D9001BC1DB81DA1B
:10363000401A001EC1DE81DF401F01DDC01D801C5D
:1036400041DC0014C1D481D5401501D7C0178016C4
:1036500041D601D2C012801341D30011C1D181D013
:10366000401001F0C030803141F10033C1F381F2EC
:1036700040320036C1F681F7403701F5C03580345D
:1036800041F4003CC1FC81FD403D01FFC03F803E54
:1036900041FE01FAC03A803B41FB0039C1F981F893
:1036A00040380028C1E881E9402901EBC02B802A7D
:1036B00041EA01EEC02E802F41EF002DC1ED81ECDB
:1036C000402C01E4C024802541E50027C1E781E6C4
:1036D00040260022C1E281E3402301E1C021802095
:1036E00041E001A0C060806141A10063C1A381A24B
:1036F00040620066C1A681A7406701A5C0658064DD
:1037000041A4006CC1AC81AD406D01AFC06F806E53
:1037100041AE01AAC06A806B41AB0069C1A981A812
:1037200040680078C1B881B9407901BBC07B807A1C
:1037300041BA01BEC07E807F41BF007DC1BD81BC5A
:10374000407C01B4C074807541B50077C1B781B6C3
:1037500040760072C1B281B3407301B1C071807014
:1037600041B00050C190819140510193C0538052AB
:1037700041920196C056805741970055C19581945A
:103780004054019CC05C805D419D005FC19F819E53
:10379000405E005AC19A819B405B0199C059805894
:1037A00041980188C04880494189004BC18B818A7A
:1037B000404A004EC18E818F404F018DC04D804CDC
:1037C000418C0044C184818540450187C0478046C3
:1037D00041860182C042804341830041C181818092
:1037E0004040000004380008000000208C00000069
:1037F000A02C0008903800088C000020B444000081
:10380000B02C0008000000000000000000000000D4
:1038100000000000000000000000000000000000A8
:103820000000000000000000000000000000000098
:103830000000000000000000000000000000000088
:103840000000000000000000000000000000000078
:10385000000000000000000000000000010203045E
:1038600001020304060708090204060800366E0177
:103870000000000000000000010203040607080920
:103880000000000000000000000000000000000038
:0400000508000131BD
:00000001FF
